:103DFC000FC30FBF0FBB0FB60FB20FAC0FA70FA1A6
:103E0C000F9B0F950F8E0F870F800F780F700F6819
:103E1C000F5F0F550F4B0F410F360F2B0F1F0F124C
:103E2C000F060EF80EEA0EDB0ECC0EBC0EAB0E9A85
:103E3C000E880E750E620E4E0E390E240E0E0DF7F8
:103E4C000DDF0DC70DAE0D940D790D5E0D410D24DA
:103E5C000D070CE80CC90CA90C890C680C460C233A
:103E6C000C000BDC0BB80B930B6E0B480B210AFAF6
:103E7C000AD30AAC0A840A5B0A330A0A09E109B7B5
:103E8C00098E0965093B091108E808BE0895086CFC
:103E9C000842081907F107C807A007780750072937
:103EAC00070206DB06B5068F066A0645062105FDE8
:103EBC0005DA05B70595057405530532051204F3AB
:103ECC0004D404B60498047B045F04430428040D52
:103EDC0003F303DA03C103A90391037A0363034DCC
:103EEC0003370322030E02F902E602D302C002AE2C
:103EFC00029C028B027A026A025A024B023C022D8D
:103F0C00021F0211020301F601E901DD01D001C516
:103F1C0001B901AE01A30198018E0184017A0171EE
:103F2C000168015F0156014D0145013D0135012E2E
:103F3C000126011F01180111010B010400FE00F8FC
:103F4C0000F200EC00E600E100DC00D600D100CC71
:103F5C0000C800C300BE00BA00B600010C01010489
:103F6C0002011E030A9604013205040406006407CC
:103F7C00010108000009015A0E01010F0001120095
:103F8C006413010114013C1501FA1664FA17FFFFC2
:103F9C001D00072000072400022701012F013C30DF
:103FAC0002023201033500023603073CFFFF3DFFDE
:103FBC00FF180002191E461A00021B00022D32C8FF
:103FCC002E0001FAFAFA18000019FFFF1A00001B64
:103FDC0000002D32C82E0001FAFAFA18000019FF61
:103FEC00FF1A00001B00002DFFFF2EFFFFFAFAFA4C
:10004800900786E0FEA3E0FF7457BE0010D39F40E0
:100058000C903F6612001EE493F599804C900014B2
:10006800E0D394044014900786E0FEA3E0FF903F9D
:100078006612001EE493F599802F900014E0D39443
:10008800034014900786E0FEA3E0FF903F7B120038
:100098001EE493F5998012900786E0FEA3E0FF9096
:1000A8003F9012001EE493F59990078612000E9077
:1000B8000786E0FEA3E0FF746C6F4E7003751300B3
:1000C80022900072E0B402087401900072F0D20C21
:1000D80090013AE090002AF090013BE090002BF06C
:1000E80090013CE090002CF0A20AB3401690013A2F
:1000F800E0700C90013BE0700690013CE0600280EB
:1001080002C20A90013AE0B4300F90013BE0B447D4
:100118000890013CE0643B60028004D20B8002C27C
:100128000BE558B40102800302024B900057E0F53A
:1001380067900062E0F569900063E0F56A900074EA
:10014800E0F56B90007AE0900029F090007CE0F5F3
:100158006690007DE0F568900080E0F5659000818C
:10016800E0F564900090E0900041F0900091E090FC
:100178000042F0900092E0900043F0900093E090ED
:100188000044F0900094E0900045F0900095E090D5
:100198000046F0900096E0900047F0900097E090BD
:1001A8000048F0900099E0900033F090009AE090B9
:1001B8000034F090009BE0900035F090009CE090B7
:1001C8000036F0900079E0B4011790000A740FF03F
:1001D800A374FFF090000CE4F0A3F074029000798F
:1001E800F0900079E0B4035990000CE0FEA3E0FF22
:1001F80090000AE0FCA3E0FD120003741012415CB9
:10020800740812414EEF900026F0EF700674FF90CC
:100218000026F07400900079F090000BE090002721
:10022800F090000AE0900028F0900026E0900789FE
:10023800F0900027E090078AF0900028E090078B64
:10024800F0803F900081E07006755801756400A247
:100258000AB3402E90013AE090002AF090013BE06A
:1002680090002BF090013CE090002CF090002AE0E8
:10027800700C90002BE0700690002CE06002800269
:10028800C20AE5677003756702E56970037569025C
:100298007E877FA4E5678E048F05FF12413E8C3967
:1002A8008D3AE56A75F0FAA4FFAEF0E5698E048F21
:1002B80005FF12413E8C3D8D3E90004FE0F5619068
:1002C800004DE0FE900069E0B5061890004CE0FE95
:1002D800900068E0B5060C90004BE0FE900059E0F5
:1002E8006E606F900069E07006900068E0600674C8
:1002F80000900059F0900069E0B402089000497439
:1003080001F08005900049E4F0900068E0B402082C
:1003180090004A7401F0800590004AE4F09000686B
:10032800E0600690004AE060028005756103800382
:10033800756104E559B55802D20C900068E0900048
:100348004CF0900069E090004DF0900059E090006A
:100358004BF0740190009EF0740190009FF07400BF
:100368009000A0F074009000A1F074009000A2F03A
:1003780074009000A3F074009000A4F07401900041
:10038800A5F074019000A6F074009000A7F0740026
:100398009000A8F074009000A9F074009000AAF0F2
:1003A80074009000ABF074019000ACF07401900000
:1003B800ADF074009000AEF074009000AFF07400DF
:1003C8009000B0F074009000B1F074009000B2F0AA
:1003D8007401900362F07401900363F07400900359
:1003E80064F07401900365F07400900366F0740083
:1003F800900367F07400900368F074009003A2F013
:1004080074019003A3F074009003A4F074019003A6
:10041800A5F074009003A6F074009003A7F0740090
:100428009003A8F074009003E2F074009003E3F0E6
:1004380074009003E4F074019003E5F074009003F5
:10044800E6F074009003E7F074009003E8F074019C
:10045800900422F07400900423F07401900424F0B6
:100468007401900425F07400900426F07400900440
:1004780027F07400900428F022E5B554F7F5B5E5A7
:10048800B554FDF5B5C2A2D297C2A1C292C207E582
:10049800B554FBF5B5755104E55104F55290004F7C
:1004A800E0F561900025E4F0C209E5B554FEF5B524
:1004B80022750A00750900AE09AF0A7457BE000319
:1004C8009F5003020576903F6612001EE493900049
:1004D8004E1241740FBF00010EE0FC903F661200FF
:1004E8001EECFEE493FFEEC39F5026AE09AF0A0F41
:1004F800BF00010E903F6612001EAE09AF0AE493DA
:10050800FC903F6612001EE49390004E124174EC7A
:10051800F0AE09AF0A903F6612001EE49390004EB9
:10052800124174E0FC903F6812001EECFCE493FD5D
:10053800ECD39D4019903F6812001EE493FC903F55
:100548006612001EE49390004E124174ECF0AE095E
:10055800AF0A74022FFF50010E8E098F0A780A74B1
:100568000126F6500418E436F640030204BF22754B
:100578000A00750900AE09AF0A7415BE00039F5042
:1005880003020644903FBD12001EE49390004E12F1
:1005980041740FBF00010EE0FC903FBD12001EEC3D
:1005A800FEE493FFEEC39F5026AE09AF0A0FBF00CB
:1005B800010E903FBD12001EAE09AF0AE493FC90F5
:1005C8003FBD12001EE49390004E124174ECF0AE51
:1005D80009AF0A903FBD12001EE49390004E1241ED
:1005E80074E0FC903FBF12001EECFCE493FDECD3DA
:1005F8009D4019903FBF12001EE493FC903FBD122E
:10060800001EE49390004E124174ECF0AE09AF0A5C
:10061800740F6F4E7006750A15750900AE09AF0A9A
:1006280074022FFF50010E8E098F0A780A74012672
:10063800F6500418E436F6400302057D22750A00D8
:10064800750900AE09AF0A7415BE00039F50030276
:100658000712903FD212001EE49390004E1241748C
:100668000FBF00010EE0FC903FD212001EECFEE42A
:1006780093FFEEC39F5026AE09AF0A0FBF00010ECD
:10068800903FD212001EAE09AF0AE493FC903FD20D
:1006980012001EE49390004E124174ECF0AE09AFC4
:1006A8000A903FD212001EE49390004E124174E06B
:1006B800FC903FD412001EECFCE493FDECD39D406B
:1006C80019903FD412001EE493FC903FD212001EF2
:1006D800E49390004E124174ECF0AE09AF0A740F27
:1006E8006F4E7006750A15750900AE09AF0A7402D7
:1006F8002FFF50010E8E098F0A780A740126F650D2
:100708000418E436F6400302064B22750A00750900
:1007180000AE09AF0A7415BE00039F50030207E03C
:10072800903FE712001EE49390004E1241740FBFF1
:1007380000010EE0FC903FE712001EECFEE493FF80
:10074800EEC39F5026AE09AF0A0FBF00010E903FBF
:10075800E712001EAE09AF0AE493FC903FE71200CF
:100768001EE49390004E124174ECF0AE09AF0A906B
:100778003FE712001EE49390004E124174E0FC9093
:100788003FE912001EECFCE493FDECD39D40199068
:100798003FE912001EE493FC903FE712001EE49329
:1007A80090004E124174ECF0AE09AF0A740F6F4E10
:1007B8007006750A15750900AE09AF0A74022FFF95
:1007C80050010E8E098F0A780A740126F650041813
:1007D800E436F6400302071922054D22054C22058E
:1007E8004EC2CF2290F800E4936406600280FE7542
:1007F800840175A70075FF80900788E4F075C9101B
:1008080075A70F75A1C775A70075D90075CEFF75B7
:10081800A70F75F1FE75F2FF75F33775F47C75A4B3
:10082800BA75A5FF75A60775AE0075AFFF75D481BB
:1008380075D5FF75D6FF75D7FFC296C295C2A0C2FF
:100848000DC297E5B554BFF5B5E5B554DFF5B5E587
:10085800B554EFF5B5E5B5547FF5B5E5B554F7F5FD
:10086800B5E5B554FDF5B575A70075A20175A147A5
:1008780075F80975BC0175BE0475BD6C75BE077544
:10088800BDA075BE0875BD0175BC0075BB1875BCEB
:100898002075BA0875E88075D11375A70F75E1053D
:1008A80075E20075C740759700759780740A124104
:1008B8002E7597C0E5975420700280F8758F0275E1
:1008C800A700D2AF75980075A90C75A70F75AB4333
:1008D80075ADFB75AC1E75A700758911758E007511
:1008E8008C00758A00D2A9D28C758D00758B00D2C8
:1008F800ABD28E75CD0075CC0075CA0075CB00D211
:10090800ADC2CFD2CA7591047592007593CD75EFBB
:100918000675D94075CF01900786E4F0A3F07513EA
:1009280000751400C299D20A74C8F5187517001218
:10093800272575A70FE5FB90001AF0E5FA90001B34
:10094800F0E5F990001CF075A70090F800E493F525
:100958000812285C122D96900789E0900026F090E6
:10096800078AE0900027F090078BE0900028F0902D
:10097800078CE0900029F090078DE0F56790078ECE
:10098800E0F56990078FE0F56A900790E0F56B90C5
:100998000791E0F566900792E0F568900793E0F517
:1009A80065900794E0F564900795E090002AF09030
:1009B8000796E090002BF0900797E090002CF090BD
:1009C8000798E0900041F0900799E0900042F0907D
:1009D800079AE0900043F090079BE0900044F09065
:1009E800079CE0900045F090079DE0900046F0904D
:1009F800079EE0900047F090079FE0900048F09035
:100A080007A0E0900033F09007A1E0900034F09048
:100A180007A2E0900035F09007A3E0900036F0744C
:100A280000900082F090013AE0700C90013BE07079
:100A38000690013CE060028004C20A8002D20A905B
:100A4800F807E493900021F0900021E0440A900018
:100A580021F0900021E054FE900021F074069000EF
:100A680012F07402900013F090F802E493900014CE
:100A7800F07403900015F07403900016F074299038
:100A88000017F07405900018F0900014E0B4040604
:100A98007404900018F0900014E0B40306740390F6
:100AA8000018F07404900019F090F804E493900092
:100AB8001DF0740090001EF090F805E49390001F5C
:100AC800F090F806E493900020F074FF900022F074
:100AD8007453900125F07475900126F074629001AA
:100AE80027F07461900128F07472900129F07475F0
:100AF80090012AF0742090012BF0743490012CF0AE
:100B0800744590012DF0744190012EF074549001B9
:100B18002FF07420900130F07434900131F0745348
:100B2800900132F07450900133F090007AE0D39441
:100B3800014006740090007AF075580175590174E7
:100B48000390004CF01200C91204B9900014E0B4EC
:100B580004051206458011900014E0D39404400562
:100B68001205778003120713122751E5B554FEF5D5
:100B7800B5900025E4F0900786E4F0A3F075240012
:100B8800752300754800752A007529007549007598
:100B98003200753100754A00755400755500755A54
:100BA8000075510475520175343C75330075710038
:100BB8007570007572CD75560075570075430075D0
:100BC8004400754500754600755B00754700754221
:100BD80000754100900006E4F0A3F0900008E4F0EE
:100BE800A3F0755F0075600090000E74FDF0A374AB
:100BF800E8F0900023E4F07464900024F0C200D27E
:100C080001C202D203754D00756E00C294C293C230
:100C180087C290C291C20C7E017F00900028E0122A
:100C2800415C900027E02FFF50010E90000AEEF083
:100C3800A3EFF0900026E0700674FF900026F09075
:100C4800000AE0FEA3E0FFEFD394FFEE940F400705
:100C580090000AE4F0A3F07400900071F074009022
:100C68000079F07400900082F0740090008DF074A8
:100C7800009000B4F0E5687003756804743A900752
:100C88004EF074FD90074FF09003D4E0900414F0F8
:100C9800D2B0D2B7D2A7D2A6D2B1D2A3C207A2B637
:100CA800B39204A2B3B39205D29CD2EC75CF01A241
:100CB80098B34005C2981230FAE5136006A299B3BA
:100CC800B340028005C299123670E51464016005CC
:100CD800E514B4040280D5E54DD39405400CE55ADB
:100CE800C394C85002055A754D00E572C394F0507C
:100CF8001A787012003FAE70AF71EFD394E8EE949B
:100D08000340080572757100757000C28E7E047FFD
:100D180000E54C12415CE58D75F004A4FDACF0EFE4
:100D28002DFDEE3CFCE58B75F04084FF7E00ED2F39
:100D3800FFEC3EFE8E258F26D28EA2B6300401B37C
:100D48005003020E7AA2B6300401B35003020E7AA1
:100D5800A2B6405A0554E5B54401F5B5900024E41F
:100D6800F0E554D3956740447C877DA4123FFC8E00
:100D7800238F24E5482FFF50010E740112414E8E37
:100D8800238F24852448755401C28E758D00758B78
:100D980000754C00D28E7403BE00039F500690006D
:100DA800257401F0E543B40603754300D204A2B6E6
:100DB800B35003020E7AC20490006BE06018123739
:100DC800B1A200B34008E5B54408F5B58006E5B51D
:100DD80054F7F5B58002C20090006EE06018123931
:100DE80006A202B34008E5B54402F5B58006E5B5AC
:100DF80054FDF5B58006E5B554FDF5B5A207B34039
:100E080004D2878002C287900059E06004D29080A3
:100E180002C29090004AE0B40104D2948002C294C5
:100E2800900049E0B40104D2938002C293A209B3AE
:100E38004004D2918002C291900018E0FE90001404
:100E4800E0C39E4009900014E0D39408400974FB65
:100E5800900023F012048190001DE0601590001DA1
:100E6800E0FE900017E06E600974FE900023F01217
:100E78000481C2CA7E017F00E54E12415CE5CD2F98
:100E8800FF50010E8E278F28D2CAE566B40148901C
:100E9800000EE0FCA3E0FDEFC39DEE9C4039B208D4
:100EA800E52A45296013A208B34008E5B54404F5CE
:100EB800B58006E5B554FBF5B590000EE0FEA3E05D
:100EC800FF900010E0FCA3E0FDEF2DFDEE3CFC9050
:100ED800000EECF0A3EDF0A2B3300501B35003020D
:100EE8000FBFA2B3300501B35003020FBFA2B35026
:100EF80003020FB80555E5B54401F5B5900024E4A3
:100F0800F0E555D395695003020FB67CEA7D60AED3
:100F180027AF28123FFC8E298F2AE56A12415C749C
:100F2800FF8E048F05FF12413E8C298D2AE5492D3D
:100F3800FD50010C74018C068D0712414E8E298FCD
:100F48002A852A49A209B34015746412415C9000AD
:100F580067E08E048F05FF12413E8C298D2A755556
:100F68000190000EE0FEA3E0FFAC27AD28120003BD
:100F780090000EEEF0A3EFF0E568FF12413E740A10
:100F8800FF12413E90007BE08C068D0712415C7495
:100F9800148E048F05FF12413E900010ECF0A3ED73
:100FA800F0C2CA75CD0075CC00754E00D2CAD20504
:100FB800A2B3B34002C205900025E0B40107E5568C
:100FC800C3940640030215D0E56E902704F828283C
:100FD80073900059E0C39402400302112DE551D3E8
:100FE8009401500302112DE55175F040A4FFAEF0B5
:100FF80090031212001EE0C395455018E55175F094
:1010080040A4FFAEF090031112001EE0F52E752DDE
:101018000002112DE55175F040A4FFAEF0900310C9
:1010280012001EE0C3954540030210C9E55175F052
:1010380040A4FFAEF090031112001EE55175F04078
:10104800A4FFAEF0E0FC90030F12001EECFEE0FFE0
:10105800EEC39FFEE5518E0475F040A4FFAEF090FC
:10106800031012001EE0F40425458C0088F0A4FF4C
:10107800AEF0E5518F048E0575F040A4FFAEF090F8
:10108800031212001EE55175F040A4FFAEF0E0FA1D
:1010980090031012001EEAFEE0FFEEC39FFECDCCC7
:1010A800CD8E0712413EE55175F040A4FFAEF09099
:1010B800030F12001EE02DFD50010C8C2D8D2E808B
:1010C80064E55175F040A4FFAEF090030F12001EC6
:1010D800E55175F040A4FFAEF0E0FC90030E12005D
:1010E8001EECFEE0FFEEC39F8545F0A4FFAEF0E5E1
:1010F800518F048E0575F040A4FFAEF090031012D6
:10110800001EE0FECDCCCD8E0712413EE55175F0B4
:1011180040A4FFAEF090030E12001EE02DFD50011A
:101128000C8C2D8D2E756E010215D0900059E0C3E0
:10113800940240030212E090004FE0D3955150030F
:10114800021289E55175F040A4FFAEF09003181221
:10115800001EE0C395455018E55175F040A4FFAE58
:10116800F090031712001EE0F52C752B000212896F
:10117800E55175F040A4FFAEF090031612001EE092
:10118800C395454003021225E55175F040A4FFAE12
:10119800F090031712001EE55175F040A4FFAEF061
:1011A800E0FC90031512001EECFEE0FFEEC39FFE6C
:1011B800E5518E0475F040A4FFAEF09003161200BE
:1011C8001EE0F40425458C0088F0A4FFAEF0E5513C
:1011D8008F048E0575F040A4FFAEF090031812003E
:1011E8001EE55175F040A4FFAEF0E0FA9003161228
:1011F800001EEAFEE0FFEEC39FFECDCCCD8E0712A7
:10120800413EE55175F040A4FFAEF0900315120081
:101218001EE02DFD50010C8C2B8D2C8064E5517542
:10122800F040A4FFAEF090031512001EE55175F0D2
:1012380040A4FFAEF0E0FC90031412001EECFEE0A8
:10124800FFEEC39F8545F0A4FFAEF0E5518F048EF5
:101258000575F040A4FFAEF090031612001EE0FEE4
:10126800CDCCCD8E0712413EE55175F040A4FFAEBE
:10127800F090031412001EE02DFD50010C8C2B8DF4
:101288002CE551B40122E561D39401401BE551C31B
:1012980095565014E545C39405500D90035FE0A89A
:1012A80029B80006952A40028003755102E551B518
:1012B800612290004FE0D395514019E55175F040F7
:1012C800A4FFAEF090031712001EE0A823B8000692
:1012D8009524400280020561756E020215D09000C7
:1012E80059E0B4022AE55175F040A4FFAEF090032E
:1012F8001712001EE0F52C752B00E55175F040A47F
:10130800FFAEF090030E12001EE0F52E752D009032
:101318000059E0B4030F900051E0F52C752B0075CF
:101328002E00752D00756E030215D0E55175F0403D
:10133800A4FFAEF090032012001EE0C3955A4003AC
:10134800021407900049E07036E551D39401402912
:10135800AE23AF24AC2DAD2EEDD39FEC9E401AE505
:101368005175F040A4FFAEF090031E12001EE0A8D5
:1013780029B80005D3952A5002800215518034E51A
:1013880051D394024029AE23AF24AC2DAD2EEDD31A
:101398009FEC9E401AE55175F040A4FFAEF0900313
:1013A8001E12001EE0A829B80005D3952A50028015
:1013B800021551E551B55236E551C39561502FE5F7
:1013C80051C395565028AE23AF24AC2BAD2CEFD388
:1013D8009DEE9C4019E55175F040A4FFAEF09003D6
:1013E8001F12001EE0A829B80006952A40028002B4
:1013F8000551C292E55165526005C207755A0075DC
:101408006E040215D0E55175F040A4FFAEF09003CC
:101418001A12001EE0B40117E55175F040A4FFAEA2
:10142800F090032012001EE0240AC3955A400302DC
:1014380014DD753064752F00A207B3500B9000605F
:10144800E02405C3954540030214DDE55175F040DD
:10145800A4FFAEF090031D12001EE0C39545406442
:10146800E55175F040A4FFAEF090031C12001EE594
:101478005175F040A4FFAEF0E0FC90031B12001E73
:10148800ECFEE0FFEEC39F8545F0A4FFAEF0E5510A
:101498008F048E0575F040A4FFAEF090031D120076
:1014A8001EE0FECDCCCD8E0712413EE55175F040D1
:1014B800A4FFAEF090031B12001EE02DFD50010C9E
:1014C8008C2F8D30AE23AF24AC2FAD30EFD39DEEF3
:1014D8009C4002D207756E050215D0E551B401098A
:1014E800900059E0C3940240030215B0900358E0FD
:1014F800D3954550030215B0900356E0C395455067
:1015080040900357E0FE900355E0F4042EFE90034C
:1015180056E0F40425458E0088F0A4FFAEF0900351
:1015280058E0FC900356E0F4042C8E048F05FF125B
:10153800413E900355E02DFD50010C8C2B8D2C80E5
:101548002C900355E0FE900354E0F4042E8545F0FA
:10155800A4FFAEF0900356E08E048F05FF12413EC3
:10156800900354E02DFD50010C8C2B8D2CE551C3BC
:101578009561502FE551C395565028AE23AF24AC42
:101588002BAD2CEFD39DEE9C4019E55175F040A48E
:10159800FFAEF090031F12001EE0A829B8000695C0
:1015A8002A40028003755102900049E0B40106E523
:1015B80051640160028003755102E551655260056E
:0815C800C207755A00756E00A0
:10270400020FD90211330212E602133302140D022E
:0227140014E3CC
:1015D000900050E02402A823B80007D395244002CD
:1015E000C207900025E0B40109900059E0C39403BC
:1015F0004003021756900049E060030216A6E55129
:10160000D394014034E55175F040A4FFAEF090034F
:101610001412001EE0A823B8001FD39524401AE539
:101620005175F040A4FFAEF090031F12001EE0A819
:1016300029B80005D3952A500280021551E551D3EF
:101640009401402FE55175F040A4FFAEF0900312D5
:1016500012001EE0C39545501AE55175F040A4FFF5
:10166000AEF090031E12001EE0A829B80005D39525
:101670002A500280021551E551D394014021E551D1
:10168000D39556401AE55175F040A4FFAEF0900393
:101690001E12001EE0A829B80005D3952A5002802A
:1016A00002155102174BE551D394024034E55175B0
:1016B000F040A4FFAEF090031412001EE0A823B87F
:1016C000001FD39524401AE55175F040A4FFAEF0F9
:1016D00090031F12001EE0A829B80005D3952A50D8
:1016E0000280021551E551D39402402FE55175F067
:1016F00040A4FFAEF090031212001EE0C3954550C7
:101700001AE55175F040A4FFAEF090031E12001EC2
:10171000E0A829B80005D3952A500280021551E5AA
:1017200051D394024021E551D39556401AE55175A5
:10173000F040A4FFAEF090031E12001EE0A829B8EE
:101740000005D3952A500280021551E5516552607B
:1017500005C207755A00900060E0D3954550099086
:101760000054E0C395455002C207900059E0700351
:101770000219B9A2A5B34008A2A4B340030219A25A
:10178000AE35AF367441D39F749C9E4005783512B8
:10179000003FAE35AF36EFB48806EEB413028003D7
:1017A00002197FA2A55003021842900059E0B4012B
:1017B0000B90004FE0D3956140020561900059E025
:1017C000B40253E55175F040A4FFAEF0900320122F
:1017D000001EE0C3955A503E90004FE0D395514013
:1017E00020E551C395565019E55175F040A4FFAE60
:1017F000F090031412001EE0A823B80006952440C0
:10180000028002055190004FE0F561E5516552609C
:1018100005C207755A00900059E0B4032590004FA7
:10182000E0D395514007E551C3955640028002052B
:101830005190004FE0F561E55165526005C20775B2
:101840005A00A2A4500302197F900059E0B4016E1F
:10185000900049E07035E551D394014029E5517578
:10186000F040A4FFAEF090031E12001EE0A829B8BD
:10187000000FD3952A400A1551755A008551618091
:101880000385516180037561018033E551D3940272
:101890004029E55175F040A4FFAEF090031E120000
:1018A0001EE0A829B8000FD3952A400A1551755A91
:1018B000008551618003855161800375610290004C
:1018C00059E0D394015003021973E55175F040A417
:1018D000FFAEF090032012001EE0C3955A400302B1
:1018E0001973900049E07041E551D394014034E50B
:1018F0005175F040A4FFAEF090031112001EE0A855
:1019000023B8001FD39524401AE55175F040A4FF79
:10191000AEF090031E12001EE0A829B80005D39572
:101920002A500280021551803FE551D39402403481
:10193000E55175F040A4FFAEF090031112001EE0D7
:10194000A823B8001FD39524401AE55175F040A490
:10195000FFAEF090031E12001EE0A829B80005D3C8
:10196000952A500280021551E55165526005C20763
:10197000755A00E556B40704055F8003755F00E5FE
:1019800064B4010EAE35AF36EF64407005EE649C72
:101990006002800EA2A54003755801A2A440037501
:1019A0005802A2A5B3B35006A2A4B3B34002800666
:1019B000753600753500021AA7A2A5B34008A2A487
:1019C000B34003021A93AE35AF367441D39F749C73
:1019D0009E4005783512003FAE35AF36EFB488062D
:1019E000EEB413028003021A93A2A5406F90006820
:1019F000E0605A90004AE0B4010790004AE4F080A9
:101A00000690004A7401F090004AE0700575610389
:101A1000800375610490004AE0B40104D29480020E
:101A2000C294E551B4041AE55175F040A4FFAEF03C
:101A300090031E12001EE0A829B80005D3952A5075
:101A4000028008755103C207755A0080037561044E
:101A5000E556B40704055F8003755F00A2A4403318
:101A6000900069E06021900049E0B40107900049CE
:101A7000E4F080069000497401F0900049E0B40160
:101A800004D2938002C293E556B40704055F800335
:101A9000755F00A2A5B3B35006A2A4B3B340028001
:101AA00006753600753500E5586559600690008268
:101AB000E06003021C2FC29C751400751300C2CA9B
:101AC000E558902716F82828738012122D96800D5D
:0D1AD000122E6F8008122F48800312302163
:0F271600021AC9021ACB021AD0021AD5021ADA15
:101ADD00900029E090007AF0E567900057F0E569F5
:101AED00900062F0E56A900063F0E56B900074F091
:101AFD00E56690007CF0E56890007DF0E56590006E
:101B0D0080F0E564900081F090002AE090013AF0B9
:101B1D0090002BE090013BF090002CE090013CF008
:101B2D00900041E0900090F0900042E0900091F024
:101B3D00900043E0900092F0900044E0900093F00C
:101B4D00900045E0900094F0900046E0900095F0F4
:101B5D00900047E0900096F0900048E0900097F0DC
:101B6D00900033E0900099F0900034E090009AF0EE
:101B7D00900035E090009BF0900036E090009CF0D6
:101B8D007400900082F07453900125F074759001EB
:101B9D0026F07462900127F07461900128F0747240
:101BAD00900129F0747590012AF0742090012BF0AA
:101BBD00743490012CF0744590012DF07441900116
:101BCD002EF0745490012FF07420900130F0743485
:101BDD00900131F07453900132F07450900133F054
:101BED009003D4E0900414F0743A90074EF074FD15
:101BFD0090074FF01200C9900004E4F0A3F090009C
:101C0D00067475F0A37430F09000087475F0A37429
:101C1D0030F0855859D2CA754C00D29C741B900077
:101C2D0023F0E556C394065005E551B55203021C49
:101C3D00C3C207E55175F040A4FFAEF09003221228
:101C4D00001EE030E003D38001C39296E55175F09C
:101C5D0040A4FFAEF090032312001EE030E003D34A
:101C6D008001C39295E55175F040A4FFAEF090034D
:101C7D002412001EE030E003D38001C3920DE55223
:101C8D00B40306E551640260028002D2A0E552B4AD
:101C9D000206E551640160028002D2A0855152AE68
:101CAD0029AF2A7405BE00039F5007E545D394055F
:101CBD0050028002D292E556D394055003021DCDF9
:101CCD00C207E551D394014073E55175F040A4FF6F
:101CDD00AEF090031E12001EE0A829B80007D395A0
:101CED002A40021551E5516552604EE55175F0409F
:101CFD00A4FFAEF090032212001EE030E003D3806B
:101D0D0001C39296E55175F040A4FFAEF090032308
:101D1D0012001EE030E003D38001C39295E55175AA
:101D2D00F040A4FFAEF090032412001EE030E0035B
:101D3D00D38001C3920D855152021DCDE556B406D7
:101D4D00279000ACE030E003D38001C39296900061
:101D5D00ADE030E003D38001C392959000AEE0304A
:101D6D00E003D38001C3920DE556B407279000A57B
:101D7D00E030E003D38001C392969000A6E030E0FE
:101D8D0003D38001C392959000A7E030E003D38088
:101D9D0001C3920DE556B4082790009EE030E00394
:101DAD00D38001C3929690009FE030E003D3800171
:101DBD00C392959000A0E030E003D38001C3920D53
:101DCD00900072E06058E54575F00284FF7E00904A
:101DDD00014E12001EE0F55CE54775F00A84FF7EAA
:101DED000090024E12001EE0F55EE55C255ED39478
:101DFD0064400BE55C255EC39464F55C8003755C03
:101E0D0000E55C75F00284FF7E008F5CEFC39433B8
:101E1D005007EF24CDF55C8003755CFF801CE54514
:101E2D0075F00284FF7E0090014E12001EE075F0E9
:101E3D000284FF7E00EF24CDF55CE595C3955C40F3
:101E4D0004C2A28002D2A2A207B34005E556B40790
:101E5D00037572CDE595C395724004C2A18002D27F
:101E6D00A1900083E0702BE54575F00284FF7E00A4
:101E7D0090018012001EE075F00284FF7E00EF24B9
:101E8D00CDF55DE595C3955D4004D2978002C2976F
:101E9D008027900083E0B40105A2B2B34002800414
:101EAD00C2978015900083E0B40206A2B2B3B3408E
:101EBD00028004C2978002D297E543C39406400383
:101ECD000224C9A2EDB350030224C9C2EDE543605B
:101EDD000302202B7E017F00E5BE12415CE5BD2F84
:101EED00FF50010E900000EEF0A3EFF0900029E0FE
:101EFD00B401177E0F7FFF900000E0FCA3E0FD1200
:101F0D000003900000EEF0A3EFF0900079E0B40232
:101F1D005B900000E0FEA3E0FF90000AE0FCA3E070
:101F2D00FDEDD39FEC9E400F900000E0F8A3E090F4
:101F3D00000AC8F0A3C8F0900000E0FEA3E0FF90F7
:101F4D00000CE0FCA3E0FDEFD39DEE9C400F900054
:101F5D0000E0F8A3E090000CC8F0A3C8F0900000DA
:101F6D00E0FEA3E0FF740412414E8F44900079E02F
:101F7D007060900000E0FEA3E0FF90000AE0FCA37B
:101F8D00E0FDEFD39DEE9C400D120003900000EE9E
:101F9D00F0A3EFF08007900000E4F0A3F0900000B4
:101FAD00E0FEA3E0FF741012415C900026E08E0469
:101FBD008F05FF12413E900000ECF0A3EDF0740090
:101FCD00D39D74019C4008900001E0F54480037599
:101FDD0044FFE54475F00AA4FFAEF074198E048F2A
:101FED0005FF12413E8D45ED2532FFAE3150010EFC
:101FFD00740112414E8F45854532753100EFD394F2
:10200D00624003754562900072E0640160069000C5
:10201D0066E060028005754301800375BB17E543DB
:10202D00B40102800302211B7E017F00E5BE124137
:10203D005CE5BD2FFF50010E900000EEF0A3EFF018
:10204D00900072E0B4017EE53445336025AC33ADCC
:10205D00341DBDFF011C8F028E038C068D07903D34
:10206D00FC12002EE493FE740193FFEFC39AEE9BD6
:10207D00400280057833124186AE33AF3474B3BE5F
:10208D000025D39F4021900000E0FCA3E0FD0FBF91
:10209D0000010E903DFC12002EE493FE740193FF9F
:1020AD00EDC39FEC9E40028005783312003FAE33A6
:1020BD00AF34E56B12415C74648E048F05FF1241E1
:1020CD003E8D478033900066E0602D900000E0FE6D
:1020DD00A3E0FFEFD39400EE9408400F900066E06C
:1020ED00B40104C2098002D209800D900066E0B4EB
:1020FD000104D2098002C209900072E064026006F8
:10210D00900066E0600575BB168003754302E543DC
:10211D00B4020280030222097E017F00E5BE124156
:10212D005CE5BD2FFF50010E900000EEF0A3EFF027
:10213D00900072E0B4027EE53445336025AC33ADDA
:10214D00341DBDFF011C8F028E038C068D07903C44
:10215D009212002EE493FE740193FFEFC39AEE9B4F
:10216D00400280057833124186AE33AF3474B3BE6E
:10217D000025D39F4021900000E0FCA3E0FD0FBFA0
:10218D0000010E903C9212002EE493FE740193FF19
:10219D00EDC39FEC9E40028005783312003FAE33B5
:1021AD00AF34E56B12415C74648E048F05FF1241F0
:1021BD003E8D478033900066E0602D900000E0FE7C
:1021CD00A3E0FFEFD39400EE9408400F900066E07B
:1021DD00B40104C2098002D209800D900066E0B4FA
:1021ED000104D2098002C209900072E070037547A4
:1021FD0000900066E07002C20975BB1FE543B40391
:10220D00457E017F00E5BE12415CE5BD2FFF50010B
:10221D000E900000EEF0A3EFF0740912415C74E62D
:10222D008E048F05FF12413E8C418D42E54A2DFDF6
:10223D0050010C74018C068D0712414E8E418F4258
:10224D0085424A75BB19E543B4040280030223B1EC
:10225D007E017F00E5BE12415CE5BD2FFF50010EF2
:10226D00900000EEF0A3EFF0740412414E8F4BE599
:10227D0065B40102800302233E756C00756C00E5A8
:10228D006CD39407400302232BE56C90004112415F
:10229D0074E0D3954B501AE56C900041124174E0F7
:1022AD00F404254BFEE56C900037124174EEF0807E
:1022BD0017E56C900041124174E0C3954BFEE56C3F
:1022CD00900037124174EEF0E56CC3940440099010
:1022DD000084E0C3956C503BE56C6029E56C900083
:1022ED0037124174FEE0FFEE90003FE0D39F4013A4
:1022FD00E56C900037124174E090003FF0E56C9072
:10230D000040F0800E900037E090003FF074009098
:10231D000040F0786C740126F6400302228C900088
:10232D0040E0F4042408F556E556D394054002C266
:10233D0092E565D39401402FE54BD3946E4004D2C2
:10234D000E8002C20E755605E565B40205A20EB3E8
:10235D0040028003755607E565B40306A20EB3B3BC
:10236D0040028003755607E55765566008E5510430
:10237D00F552855657E556B40708E5B54480F5B5D1
:10238D008006E5B5547FF5B5E55664066005E5565E
:10239D00B40808E5B54410F5B58006E5B554EFF57C
:1023AD00B575BB13E543B4050280030224C57E0158
:1023BD007F00E5BE12415CE5BD2FFF50010E900080
:1023CD0000EEF0A3EFF0740412414E8F46E564B4B5
:1023DD00020280030224C2756C00756C00E56CD39B
:1023ED0094034003022479E56C900033124174E0AC
:1023FD00D39546501AE56C900033124174E0F40405
:10240D002546FEE56C90002D124174EEF08017E527
:10241D006C900033124174E0C39546FEE56C90005C
:10242D002D124174EEF0E56C6029E56C90002D12D3
:10243D004174FEE0FFEE900031E0D39F4013E56C58
:10244D0090002D124174E0900031F0E56C90003257
:10245D00F0800E90002DE0900031F074009000326D
:10246D00F0786C740126F640030223EA900082E0B6
:10247D007043E52A45296036E558C39403500A9008
:10248D000032E004C3940340028007900032E00460
:10249D00F558E558D39402400A900032E004D394E5
:1024AD000250028007900032E004F558800790003A
:1024BD0032E004F55875BB180543D2ECE55FD394B3
:1024CD000450030225DD75CF01C2A2AE35AF3674BF
:1024DD0088D39F74139E4005A2A5B34014AE35AFAB
:1024ED00367488D39F74139E4005A2A4B340028016
:1024FD0048783512003FAE35AF36EFB4883BEEB4B9
:10250D001337A2A5B3500990004FE0D39551500257
:10251D00800405518011A2A5B3500890004FE065CD
:10252D005160028002D207A2A4B35007E551D394A3
:10253D0001500280041551C207A2A5B3B35006A2E3
:10254D00A4B3B340028006753600753500E55165BC
:10255D0052604EE55175F040A4FFAEF0900322128B
:10256D00001EE030E003D38001C39296E55175F073
:10257D0040A4FFAEF090032312001EE030E003D321
:10258D008001C39295E55175F040A4FFAEF0900324
:10259D002412001EE030E003D38001C392A08551C8
:1025AD0052900083E06005A2B2B340028004C2974E
:1025BD008002D297A20740057572CD80037572FF18
:1025CD00E595C395724004C2A18002D2A10224D325
:1025DD00AE25AF26EFD39420EE944E50030226D8AD
:1025ED00120481C28E758D00758B00754C00D28ED4
:1025FD00C2077571007570007572CD755104752423
:10260D0000752300755400755A00C287900059E07B
:10261D006004D2908002C29090004AE0B40104D2CE
:10262D00948002C294900049E0B40104D2938002D8
:10263D00C293A209B34004D2918002C29190006B63
:10264D00E060181237B1A200B34008E5B54408F5B3
:10265D00B58006E5B554F7F5B58002C20090006E61
:10266D00E06018123906A202B34008E5B54402F540
:10267D00B58006E5B554FDF5B58006E5B554FDF517
:10268D00B590000E74FDF0A374E8F0E543B40603B5
:10269D00754300900025E4F0752600752500758DB5
:1026AD0000758B00754C00900024E0C39403500816
:1026BD00900024E004F080067403900024F0900054
:1026CD0024E0B40306E5B554FEF5B5AE27AF28EF0B
:1026DD00D39410EE9427401CC2CA75CD0075CC0062
:1026ED00752800752700D2CA754E00752A00752908
:0726FD0000755500020CB44A
:103AB8000000010001320164019601960200021221
:103AC80002240200020003000340038003C0040034
:103AD8000440048004C00500060006000600060035
:103AE800060006000600060000FF0131016301958B
:103AF80001FF01FF0211022302FF02FF02FF033F41
:103B0800037F03BF03FF043F047F04BF04FF05FFD7
:103B180006FF06FF06FF06FF06FF06FF06FF06FF75
:103B28000FAA0FA50F9F0F9A0F940F8D0F870F8065
:103B38000F780F710F680F600F570F4E0F450F3B2F
:103B48000F300F250F1A0F0E0F020EF50EE80EDBC1
:103B58000ECC0EBE0EAE0E9F0E8E0E7D0E6C0E5A45
:103B68000E470E340E200E0C0DF70DE20DCB0DB5E1
:103B78000D9D0D850D6D0D540D3A0D200D050CE9AB
:103B88000CCE0CB10C940C760C580C3A0C1B0BFB9D
:103B98000BDB0BBB0B9A0B790B570B350B130AF18D
:103BA8000ACE0AAB0A870A640A400A1C09F809D433
:103BB80009B0098C09670943091F08FB08D608B230
:103BC800088E086A0846082307FF07DC07B9079626
:103BD80007730751072F070D06EC06CA06AA0689C0
:103BE80006690649062A060A05EC05CD05B00592C0
:103BF80005750558053C0520050504EA04CF04B5FC
:103C0800049C04820469045104390422040B03F45B
:103C180003DE03C803B2039D038903750361034DE3
:103C2800033B03280316030402F202E102D102C097
:103C380002B002A002910282027302650257024991
:103C4800023C022F02220216020901FD01F201E6DE
:103C580001DB01D001C601BB01B101A7019D01949F
:103C6800018B0182017901700168016001580150DE
:103C78000148014101390132012B0125011E0118BA
:103C88000111010B010500FF00FA0FA60FA00F9903
:103C98000F920F8B0F840F7C0F740F6B0F620F58EE
:103CA8000F4E0F430F380F2C0F1F0F120F050EF773
:103CB8000EE80ED80EC80EB70EA50E930E800E6C29
:103CC8000E580E420E2C0E150DFD0DE40DCB0DB148
:103CD8000D950D790D5D0D3F0D200D010CE10CC00A
:103CE8000C9E0C7C0C590C350C100BEA0BC40B9E6B
:103CF8000B760B4F0B260AFD0AD40AAA0A800A552E
:103D08000A2A09FF09D409A8097C0950092508F9D4
:103D180008CD08A10875084A081E07F307C8079DBB
:103D280007730749072006F706CE06A6067E06573C
:103D38000630060A05E405BF059B057705540532DC
:103D4800051004EF04CE04AE048F04710453043547
:103D5800041903FD03E203C703AD0394037B036364
:103D6800034B0334031E030802F302DE02CA02B641
:103D780002A30291027F026D025C024C023C022CFB
:103D8800021D020E020001F201E401D701CA01BEC0
:103D980001B101A6019A018F0185017A01700166BE
:103DA800015D0153014A0141013901310129012114
:103DB80001190112010B010400FD00F700F000EAEF
:103DC80000E400DE00D900D300CE00C900C400BF63
:103DD80000BA00B500B100AD00A800A400A0009C86
:103DE800009900950091008E008A00870084008168
:043DF800007E007BCE
:10272500751A00751900AE19AF1AAC17AD18EDC3BF
:102735009FEC9E401674FF12412E75CF01781A74D6
:102745000126F6500418E436F650DB22900786E49D
:10275500F0A3F0751000750F00751300751400C215
:102765000FD21022C2AF75D900758F0375B7A57545
:10277500B7F190F800E4F0758F0175B7A575B7F15D
:10278500E50890F800F075B7A575B7F190F801E484
:10279500F075B7A575B7F190079DE090F802F07553
:1027A500B7A575B7F19007A1E090F803F075B7A547
:1027B50075B7F190079EE090F804F075B7A575B769
:1027C500F190079FE090F805F075B7A575B7F19002
:1027D50007A0E090F806F075B7A575B7F19007A2C8
:1027E500E090F807F0758F0075D940D2AF229007B9
:1027F50088E0B4AB61C2AF75D90075B62275F52214
:10280500758F0375B7A575B7F1740090F600F0756F
:102815008F01750A00750900AE09AF0A7413BE0071
:10282500279F402475B7A575B7F190078912001E3B
:10283500E0FC90F60012001EECF0780A740126F612
:10284500500418E436F650D0758F0075F51175B63D
:102855002075D940D2AF22C2AF75D90075F5227562
:102865000A00750900AE09AF0A7413BE00229F4025
:102875001F90F60012001EE493FC90078912001EBB
:10288500ECF0780A740126F6500418E436F650D5B3
:1028950075F51175D940D2AF22900788E0B4AA0228
:1028A50080030229DBC2AF75D90075B62275F52202
:1028B500758F0375B7A575B7F1740090EE00F075C7
:1028C500B7A575B7F1740090F000F075B7A575B7A9
:1028D500F1740090F200F075B7A575B7F17400902A
:1028E500F400F0758F01750A00750900AE09AF0A8D
:1028F50074FFC39F74019E402475B7A575B7F19009
:10290500004E12001EE0FC90EE0012001EECF07866
:102915000A740126F6500418E436F650CF750A00FD
:10292500750900AE09AF0A74FFC39F74019E402468
:1029350075B7A575B7F190024E12001EE0FC90F038
:102945000012001EECF0780A740126F6500418E413
:1029550036F650CF750A00750900AE09AF0A74FF47
:10296500C39F74019E402475B7A575B7F190044EB9
:1029750012001EE0FC90F20012001EECF0780A74C2
:102985000126F6500418E436F650CF750A0075098D
:1029950000AE09AF0A74FFC39F74019E402475B74A
:1029A500A575B7F190064E12001EE0FC90F40012DA
:1029B500001EECF0780A740126F6500418E436F689
:1029C50050CF758F0075F51175B62075D940D2AF0A
:1029D500743A90074EF022900788E0B4AA0280036B
:1029E500022B19C2AF75D90075B62275F522758F00
:1029F5000375B7A575B7F1740090E600F075B7A536
:102A050075B7F1740090E800F075B7A575B7F17466
:102A15000090EA00F075B7A575B7F1740090EC0069
:102A2500F0758F01750A00750900AE09AF0A74FFCC
:102A3500C39F74019E402475B7A575B7F190004EEC
:102A450012001EE0FC90E60012001EECF0780A74FD
:102A55000126F6500418E436F650CF750A007509BC
:102A650000AE09AF0A74FFC39F74019E402475B779
:102A7500A575B7F190024E12001EE0FC90E8001219
:102A8500001EECF0780A740126F6500418E436F6B8
:102A950050CF750A00750900AE09AF0A74FFC39FD0
:102AA50074019E402475B7A575B7F190044E1200C8
:102AB5001EE0FC90EA0012001EECF0780A74012674
:102AC500F6500418E436F650CF750A00750900AEC5
:102AD50009AF0A74FFC39F74019E402475B7A5759D
:102AE500B7F190064E12001EE0FC90EC0012001E9D
:102AF500ECF0780A740126F6500418E436F650CF47
:102B0500758F0075F51175B62075D940D2AF743A39
:102B150090074EF022900788E0B4AA028003022CA9
:102B250057C2AF75D90075B62275F522758F037535
:102B3500B7A575B7F1740090DE00F075B7A575B748
:102B4500F1740090E000F075B7A575B7F1740090C9
:102B5500E200F075B7A575B7F1740090E400F07563
:102B65008F01750A00750900AE09AF0A74FFC39F8E
:102B750074019E402475B7A575B7F190004E1200FB
:102B85001EE0FC90DE0012001EECF0780A740126AF
:102B9500F6500418E436F650CF750A00750900AEF4
:102BA50009AF0A74FFC39F74019E402475B7A575CC
:102BB500B7F190024E12001EE0FC90E00012001EDC
:102BC500ECF0780A740126F6500418E436F650CF76
:102BD500750A00750900AE09AF0A74FFC39F740139
:102BE5009E402475B7A575B7F190044E12001EE0FE
:102BF500FC90E20012001EECF0780A740126F650F3
:102C05000418E436F650CF750A00750900AE09AF11
:102C15000A74FFC39F74019E402475B7A575B7F16B
:102C250090064E12001EE0FC90E40012001EECF02F
:102C3500780A740126F6500418E436F650CF758FDD
:102C45000075F51175B62075D940D2AF743A900765
:102C55004EF022900788E0B4AA028003022D95C2A7
:102C6500AF75D90075B62275F522758F0375B7A5B1
:102C750075B7F1740090D600F075B7A575B7F17406
:102C85000090D800F075B7A575B7F1740090DA001B
:102C9500F075B7A575B7F1740090DC00F0758F017C
:102CA500750A00750900AE09AF0A74FFC39F740168
:102CB5009E402475B7A575B7F190004E12001EE031
:102CC500FC90D60012001EECF0780A740126F6502E
:102CD5000418E436F650CF750A00750900AE09AF41
:102CE5000A74FFC39F74019E402475B7A575B7F19B
:102CF50090024E12001EE0FC90D80012001EECF06F
:102D0500780A740126F6500418E436F650CF750A91
:102D150000750900AE09AF0A74FFC39F74019E4098
:102D25002475B7A575B7F190044E12001EE0FC900E
:102D3500DA0012001EECF0780A740126F650041829
:102D4500E436F650CF750A00750900AE09AF0A746E
:102D5500FFC39F74019E402475B7A575B7F1900612
:102D65004E12001EE0FC90DC0012001EECF0780A0A
:102D7500740126F6500418E436F650CF758F0075A9
:102D8500F51175B62075D940D2AF743A90074EF05B
:102D950022C2AF75D90075F522750A00750900AE16
:102DA50009AF0A74FFC39F74019E401F90EE001285
:102DB500001EE493FC90004E12001EECF0780A749D
:102DC5000126F6500418E436F650D4750A00750944
:102DD50000AE09AF0A74FFC39F74019E401F90F0B7
:102DE5000012001EE493FC90024E12001EECF078D7
:102DF5000A740126F6500418E436F650D4750A0014
:102E0500750900AE09AF0A74FFC39F74019E401F88
:102E150090F20012001EE493FC90044E12001EEC8A
:102E2500F0780A740126F6500418E436F650D47585
:102E35000A00750900AE09AF0A74FFC39F74019EAD
:102E4500401F90F40012001EE493FC90064E120001
:102E55001EECF0780A740126F6500418E436F65094
:102E6500D475F51175D940D2AF22C2AF75D90075A9
:102E7500F522750A00750900AE09AF0A74FFC39FF4
:102E850074019E401F90E60012001EE493FC900022
:102E95004E12001EECF0780A740126F6500418E470
:102EA50036F650D4750A00750900AE09AF0A74FFED
:102EB500C39F74019E401F90E80012001EE493FC1E
:102EC50090024E12001EECF0780A740126F65004AA
:102ED50018E436F650D4750A00750900AE09AF0A34
:102EE50074FFC39F74019E401F90EA0012001EE408
:102EF50093FC90044E12001EECF0780A740126F63D
:102F0500500418E436F650D4750A00750900AE0968
:102F1500AF0A74FFC39F74019E401F90EC0012001E
:102F25001EE493FC90064E12001EECF0780A740124
:102F350026F6500418E436F650D475F51175D940C7
:102F4500D2AF22C2AF75D90075F522750A00750991
:102F550000AE09AF0A74FFC39F74019E401F90DE47
:102F65000012001EE493FC90004E12001EECF07857
:102F75000A740126F6500418E436F650D4750A0092
:102F8500750900AE09AF0A74FFC39F74019E401F07
:102F950090E00012001EE493FC90024E12001EEC1D
:102FA500F0780A740126F6500418E436F650D47504
:102FB5000A00750900AE09AF0A74FFC39F74019E2C
:102FC500401F90E20012001EE493FC90044E120094
:102FD5001EECF0780A740126F6500418E436F65013
:102FE500D4750A00750900AE09AF0A74FFC39F7452
:102FF500019E401F90E40012001EE493FC90064ED3
:1030050012001EECF0780A740126F6500418E43616
:10301500F650D475F51175D940D2AF22C2AF75D926
:103025000075F522750A00750900AE09AF0A74FF2F
:10303500C39F74019E401F90D60012001EE493FCAE
:1030450090004E12001EECF0780A740126F650042A
:1030550018E436F650D4750A00750900AE09AF0AB2
:1030650074FFC39F74019E401F90D80012001EE498
:1030750093FC90024E12001EECF0780A740126F6BD
:10308500500418E436F650D4750A00750900AE09E7
:10309500AF0A74FFC39F74019E401F90DA001200AF
:1030A5001EE493FC90044E12001EECF0780A7401A5
:1030B50026F6500418E436F650D4750A0075090052
:1030C500AE09AF0A74FFC39F74019E401F90DC00D8
:1030D50012001EE493FC90064E12001EECF0780AD6
:1030E500740126F6500418E436F650D475F51175BA
:1030F500D940D2AF22E51464046006E59964FF6007
:10310500028031A20F4004D20F8027E514600874B5
:10311500E62514900023F0E513600874F02513905C
:103125000023F0E514B4010280FE75140075130048
:10313500C20F8002C20FE514903A5BF82828737518
:103145001400E599B4FF03751301E599B4FE037501
:103155001302E599B4FD03751303E599B4FC0375F2
:103165001304E599B4FA03751305E599B4FB0675DF
:103175001401120481E599B4F90675140412048149
:10318500E599D394E54007E599C394F0400280168C
:103195008599157514027E017F00E515C394E61225
:1031A500415C8E0D8F0E900786E4F0A3F0E599D370
:1031B50094C44007E599C394E64002802885991593
:1031C50075140374E5C39515F50E750D00AE0DAFB9
:1031D5000E903AB812002EE493F874019390078686
:1031E500C8F0A3C8F0D29902366F900786E0FEA317
:1031F500E0FFEFC39400EE94054009EFD394FFEE92
:1032050094064013900786E0FEA3E0FF90004E125F
:10321500001EE599F0800385996D90078612000ED2
:10322500900786E0FEA3E0FFEFB40106EEB40702C7
:10323500800302347C90074EE0B43C0280030234E4
:103245007C75FFA0A20AB35005A20BB3400302335D
:103255006FC29C90007AE090078CF0900057E09048
:10326500078DF0900062E090078EF0900063E0908B
:10327500078FF0900074E0900790F090007CE0904C
:103285000791F090007DE0900792F0900080E0902B
:103295000793F0900081E0900794F090013AE09058
:1032A5000795F090013BE0900796F090013CE09087
:1032B5000797F0900090E0900798F0900091E090CB
:1032C5000799F0900092E090079AF0900093E090B3
:1032D500079BF0900094E090079CF0900095E0909B
:1032E500079DF0900096E090079EF0900097E09083
:1032F500079FF0900099E09007A0F090009AE09069
:1033050007A1F090009BE09007A2F090009CE09050
:1033150007A3F07400900082F01200C974AB900707
:0D33250088F01227F374AA900788F0E5588D
:063A5B000231440231EFCC
:10333200903A7CF8282873801212289E800D122958
:0B334200DC8008122B1A8003122C58AC
:0F3A7C0002333902333B02334002334502334AEF
:10334D00900788E4F090013AE0700C90013BE0703A
:10335D000690013CE060028004C20A8002D20A029B
:10336D003471C29C900078E0900789F090005EE087
:10337D0090078AF090005FE090078BF090007AE064
:10338D0090078CF0900057E090078DF0900062E070
:10339D0090078EF0900063E090078FF0900074E03E
:1033AD00900790F090007CE0900791F090007DE008
:1033BD00900792F0900080E0900793F0900081E0EC
:1033CD00900794F090013AE0900795F090013BE062
:1033DD00900796F090013CE0900797F0900090E0F8
:1033ED00900798F0900091E0900799F0900092E08E
:1033FD0090079AF0900093E090079BF0900094E076
:10340D0090079CF0900095E090079DF0900096E05D
:10341D0090079EF0900097E090079FF0900099E044
:10342D009007A0F090009AE09007A1F090009BE02B
:10343D009007A2F090009CE09007A3F0740090001C
:10344D0082F074AB900788F01227F374AA90078866
:10345D00F012289E1229DC122B1A122C58D29C75B0
:10346D0099FB80FED29C7514007513007599FB02B3
:10347D00366F900786E0FEA3E0FFEF4E700685994C
:10348D0010750F00900786E0FEA3E0FF74016F4EEC
:10349D00701BAC0FAD10AA0DAB0EED2BFBEC3AFA79
:1034AD008A068B0790004E12001EE599F090078654
:1034BD0012000E900786E0FEA3E0FF74026F4E70BF
:1034CD000C1200C985159975140075130002366F1D
:1034DD00900786E0FEA3E0FF90004E12001EE599D6
:1034ED00F090078612000E900786E0FEA3E0FFAC79
:1034FD000DAD0E8F028E038C068D07903AF01200E3
:10350D002EE493F9740193FEEAD39EEB994009855D
:10351D00159975140075130002366F900786E0FE3D
:10352D00A3E0FF90004E12001EE599F09007861261
:10353D00000E900786E0FEA3E0FFEFB40006EEB4A8
:10354D000102800302366F75FFA090001CE0D3943A
:10355D00C7400B90001CE0C394C8F516801A90006C
:10356D001CE0D39463400B90001CE0C39464F516EB
:10357D00800690001CE0F516E51675F002A4FFAE6E
:10358D00F08F6CEF90004E124174EFFCE0FDEC906B
:10359D000051124174EDFCE0FDEC2DB516028003D7
:1035AD000236610FEF90004E124174E56CFFE0FCA6
:1035BD00EF900052124174ECFFE0FCEFC39CB51686
:1035CD00028003023661E56C900050124174E56C87
:1035DD00FFE0FCEF900053124174ECFFE0FCEF2C88
:1035ED00B51671E56C900054124174E0C3951690B8
:1035FD00079DF0E56C900055124174E0C39516904F
:10360D00079EF0E56C900058124174E0C39516903A
:10361D00079FF0E56C900059124174E0C395169028
:10362D0007A0F0E56C90005A124174E0C395169016
:10363D0007A1F0E56C90005B124174E0C395169004
:10364D0007A2F01227697599F9751864751700129C
:10365D00272580FE7599FF751864751700122725AB
:02366D0080FEDD
:093A610002347F0234DD02352835
:10366F0022E513903A6AF82828730237B09007863C
:10367F00E0FEA3E0FF90001212001EE0F599900704
:10368F008612000E900786E0FEA3E0FF74116F4EC6
:10369F0070037513000237B08563990237B0900736
:1036AF0086E0FEA3E0FF90004E12001EE0F599EFBA
:1036BF00B40107EEB4070375130090078612000ECE
:0736CF000237B0900787E00D
:0F3A6A0002367902367C0236A70236AD0236D21A
:1036D600903A8BF82828738524990237A5852A996C
:1036E6000237A58544990237A58547990237A585EE
:1036F60051990237A58561990237A58556990237F2
:10370600A58558990237A5756F00900069E0700687
:10371600900068E060028016A2A44006E56F4404AB
:10372600F56FA2A54006E56F4402F56F801A90007A
:103736004AE0B40106E56F4410F56F900049E0B425
:103746000106E56F4420F56FA207B34006E56F4416
:1037560001F56FA209B34006E56F4408F56F856F62
:1037660099803CA210B340077599FAC2108017A23F
:103776000CB3400575990F800B900023E0F59990E6
:103786000023E4F0C20C80178542998012854B997C
:0F379600800D85469980087599FC800375130096
:103A8B000236DD0236E30236E90236EF0236F50284
:103A9B0036FB02370102370702370D02376902374F
:0D3AAB008E02379302379802379D0237A232
:0B37A50090078612000E8003120048FF
:033A79000237AD64
:1037B0002290006BE0B4010385241190006BE0B40B
:1037C0000203852A1190006BE0B403038544119035
:1037D000006BE0B4040385471190006BE0B405036F
:1037E00085511190006BE0B4060385561190006B73
:1037F000E0B4070385581190006CE0FE90006DE086
:10380000C39E500302388790006BE0D39404402C91
:1038100090006CE0D39511500990006DE0C39511B4
:1038200050028002D20090006CE0D39511500990B4
:10383000006DE0C395115002C200804990006BE01A
:10384000B4041890006DE0C395115002D2009000AE
:103850006CE0D395114002C200802A90006CE0C356
:103860009511500990006DE0D3951150028002D25D
:103870000090006CE0D39511500990006DE0C39565
:10388000115002C200807E90006BE0D39404402C63
:1038900090006CE0C39511400990006DE0D3951144
:1038A00040028002C20090006CE0C3951140099074
:1038B000006DE0D395114002D200804990006BE08A
:1038C000B4041890006CE0C395115002C20090003F
:1038D0006DE0D395114002D200802A90006CE0C3C5
:1038E0009511400990006DE0D395114002D20090EF
:1038F000006CE0D39511400990006DE0C395114034
:10390000028002C2002290006EE0B40103852411FF
:1039100090006EE0B40203852A1190006EE0B403BB
:103920000385441190006EE0B404038547119000B4
:103930006EE0B4050385511190006EE0B406038576
:10394000561190006EE0B4070385581190006FE0A7
:10395000FE900070E0C39E50030239DC90006EE0E0
:10396000D39404402C90006FE0D39511500990003F
:1039700070E0C3951150028002D20290006FE0D334
:1039800095115009900070E0C395115002C2028059
:103990004990006EE0B40418900070E0C395115097
:1039A00002D20290006FE0D395114002C202802A39
:1039B00090006FE0C395115009900070E0D395110D
:1039C00050028002D20290006FE0D395115009900E
:1039D0000070E0C395115002C202807E90006EE03C
:1039E000D39404402C90006FE0C3951140099000DF
:1039F00070E0D3951140028002C20290006FE0C3D4
:103A000095114009900070E0D395114002D20280D8
:103A10004990006EE0B4041890006FE0C395115017
:103A200002C202900070E0D395114002D202802AB7
:103A300090006FE0C395114009900070E0D395119C
:103A40004002D20290006FE0D395114009900070BF
:0B3A5000E0C3951140028002C2022278
:094174002582F582500205832228
:10002E00EF2F500205832582F582E5833E2EF58360
:01003E00229F
:08000300C3EF9DFFEE9CFE22FD
:08003F000806B60002180622B3
:0D000E00A3E004F0700612416AE004F02245
:084186000816B6FF021816220C
:0E414E00048007C3CE13CECF13CFD5E0F622E8
:103FFC00BC000FBE0008ED8FF084FFADF022E4FE94
:10400C00FF22BE000DEF60FE54F0606F20E703024C
:10401C0040B2EAC0E0EBC0E078017A0075F001EE46
:10402C0020E710EF25E0FFEE33FE0AC5F023C5F0C4
:10403C0030E7F0EA5407F9096A7A007B006001085E
:10404C00C3EC9E40167004ED9F4010ED9FFDEC9E5E
:10405C00FCE5F0CA4ACA03F5F08005E5F003F5F07B
:10406C00C3EE13FEEF13FFD9D77908CACBCAD8D049
:10407C00EAFEEBFFD0E0FBD0E0FA22EC8FF084FC00
:10408C00ED54F045F0C48FF084FEEDC454F045F0CF
:10409C00C48FF084FDEEC4FE54F02DFFEE540F3CA3
:1040AC00FEADF07C0022790078008FF0EC7E0820C9
:1040BC00E70DC3CD33CD33C933C9C833C8DEF08463
:1040CC0049F9E5F08FF0BE00E6FD7C00E9FFE8FE63
:0140DC0022C1
:0E415C00F88FF0A4FFE5F0CE88F0A42EFE222E
:10412E00600D782B024138007830D8FED5E0F822A9
:10413E00EEC0E07E00123FFCEFFDEEFCD0E0FE2272
:03000B000240DDD3
:03001B000240F8A8
:03002B000241137C
:0300000002417D3D
:09417D0075817375D0000207EC96
:0B001E00E5822FF582E5833EF583228A
:0A416A000582D5820215831582221A
:1040DD00C0E0C0F0C083C082C0D075D0001207E12F
:1040ED00D0D0D082D083D0F0D0E032C0E0C0F0C0CC
:1040FD0083C082C0D075D0001207E4D0D0D082D05A
:10410D0083D0F0D0E032C0E0C0F0C083C082C0D018
:10411D0075D0001207E7D0D0D082D083D0F0D0E098
:01412D00325F
:00000001FF
